:020000040000FA
:04080000E4EF04F02D
:1008100003B23DEF04F0F2B458EF04F09EB060EF85
:1008200004F09EB268EF04F0F2A81AEF04F0F2B2FE
:100830001CEF04F0C2EF04F0CD90F29207BC078EDB
:10084000078C9EA029EF04F00101463F29EF04F038
:10085000472B07AE34EF04F0CECF4EF1CFCF4FF1A0
:1008600046C150F147C151F1CF6ACE6A0101466BD2
:10087000476B9E90CD80C2EF04F00392030103EE1C
:1008800000F080517F0BE92604C0EFFF802B8151DF
:10089000805D700BD8A48B8200008051815D700B4D
:1008A000D8A48B9281518019D8B40790C2EF04F07C
:1008B000F2940101383FC2EF04F0392BC2EF04F08B
:1008C0009E900101463FC2EF04F0472BC2EF04F0B7
:1008D0009E92C3CF48F1C4CF49F1C28207B485EFDD
:1008E00004F03AC13EF13BC13FF13CC140F13DC192
:1008F00041F14EC152F14FC153F150C154F151C1B8
:1009000055F148C14AF149C14BF10201002FC2EF34
:1009100004F03C0E006FD57ED5BE32D0D6CF3AF172
:10092000D7CF3BF138C13CF1E86AE8CF3DF1010196
:1009300047A7A6EF04F0079C079E0101000E4E6F2B
:10094000600E4F6F3D0E506F080E516F01013ABFA0
:10095000B6EF04F03B67B6EF04F03C67B6EF04F087
:100960003D67B6EF04F0F288BBEF04F0F2984E6BEF
:100970004F6B506B516BD76AD66A0101386B396B7C
:10098000C2EF04F002C0E0FF005001C0D8FF100029
:10099000A6B2C8EF04F00CC0A9FF0BC0A8FFA69E2A
:1009A000A69CA684F29E550EA76EAA0EA76EA682DE
:1009B000F28EA694A6B2DAEF04F01200A96EA69EFB
:1009C000A69CA680A85012000F010E0EC16E800ECC
:1009D000C06E030EC26E0F01896A110E926E080E70
:1009E0008A6EF10E936E8B6A800E946EF18E0F01FB
:1009F000280ED56EF28AB00ECD6E9D8001014E6B31
:100A00004F6B506B516B526B536B546B556B566BFA
:100A1000576B586B596B079C079E760ECA6E9D826A
:100A200002013C0E006FCC6A240EAC6E0401806B98
:100A3000816B0F01900EAB6E0F019D8A0301806BDD
:100A4000816B8A6B8B920001F28EF28C07B0E8EF1B
:100A50000AF00301805181197F0BD8B4E8EF0AF046
:100A600013EE00F081517F0BE126812BE7CFE8FFE9
:100A7000E00BD8B4E8EF0AF023EE82F08A51070BBE
:100A8000D926E7CFDFFF8A2BDF50780AD8A4E8EF1A
:100A90000AF007808251720AD8B4ECEF06F0825156
:100AA000630AD8B42AEF09F08251690AD8B473EF07
:100AB00005F082517A0AD8B486EF06F05FEF09F0AC
:100AC000040114EE00F080517F0BE12682C4E7FFA1
:100AD000802B12000D0E826F60EC05F00A0E826F03
:100AE00060EC05F012000401690E826F60EC05F005
:100AF00004012C0E826F60EC05F00101030E006F03
:100B0000000E016F000E026F000E036F77EC0DF008
:100B100020C182F40401300E822760EC05F021C16F
:100B200082F40401300E822760EC05F022C182F4C9
:100B30000401300E822760EC05F023C182F4040129
:100B4000300E822760EC05F024C182F40401300EDF
:100B5000822760EC05F025C182F40401300E822763
:100B600060EC05F026C182F40401300E822760ECAF
:100B700005F027C182F40401300E822760EC05F0F5
:100B800004012C0E826F60EC05F00101030E006F72
:100B9000000E016F000E026F000E036F77EC0DF078
:100BA00020C182F40401300E822760EC05F021C1DF
:100BB00082F40401300E822760EC05F022C182F439
:100BC0000401300E822760EC05F023C182F4040199
:100BD000300E822760EC05F024C182F40401300E4F
:100BE000822760EC05F025C182F40401300E8227D3
:100BF00060EC05F026C182F40401300E822760EC1F
:100C000005F027C182F40401300E822760EC05F064
:100C100004012C0E826F60EC05F00101090E006FDB
:100C2000000E016F000E026F000E036F77EC0DF0E7
:100C300020C182F40401300E822760EC05F021C14E
:100C400082F40401300E822760EC05F022C182F4A8
:100C50000401300E822760EC05F023C182F4040108
:100C6000300E822760EC05F024C182F40401300EBE
:100C7000822760EC05F025C182F40401300E822742
:100C800060EC05F026C182F40401300E822760EC8E
:100C900005F027C182F40401300E822760EC05F0D4
:100CA00004012C0E826F60EC05F0200EF86EF76ADE
:100CB000F66A04010900F5CF82F460EC05F0090042
:100CC000F5CF82F460EC05F00900F5CF82F460EC1A
:100CD00005F00900F5CF82F460EC05F00900F5CFCE
:100CE00082F460EC05F00900F5CF82F460EC05F0C9
:100CF0000900F5CF82F460EC05F00900F5CF82F42D
:100D000060EC05F06AEC05F05FEF09F08351630ACF
:100D1000D8A45FEF09F08451610AD8A45FEF09F00D
:100D200085516C0AD8A45FEF09F08651410A2EE084
:100D30008651440A07E08651420AD8B4D9EF06F03A
:100D40005FEF09F00798079A04017A0E826F60EC52
:100D500005F00401780E826F60EC05F00401640E6A
:100D6000826F60EC05F081A8BDEF06F00401550E1E
:100D7000826F60EC05F0C2EF06F004014C0E826F4A
:100D800060EC05F06AEC05F05FEF09F00788079A60
:100D900004017A0E826F60EC05F00401410E826F4F
:100DA00060EC05F00401610E826F60EC05F0B3EFBA
:100DB00006F00798078A04017A0E826F60EC05F04E
:100DC0000401420E826F60EC05F00401610E826F37
:100DD00060EC05F0B3EF06F00401720E826F60EC78
:100DE00005F004012C0E826F60EC05F0078452C1FF
:100DF00056F153C157F154C158F155C159F13EC193
:100E000042F13FC143F140C144F141C145F14AC102
:100E10004CF14BC14DF107940101620E046F010EBC
:100E2000056F000E066F000E076F56C100F157C127
:100E300001F158C102F159C103F1DDEC0CF003BF1F
:100E400069EF07F00E0EDEEC04F0E8CF0CF10F0EA8
:100E5000DEEC04F0E8CF0DF1100EDEEC04F0E8CF8C
:100E60000EF1110EDEEC04F0E8CF0FF126EC0CF0E1
:100E700056C104F157C105F158C106F159C107F136
:100E8000DDEC0CF00782EAEC0BF026EC0CF007929C
:100E9000EAEC0BF056C100F157C101F158C102F163
:100EA00059C103F10792EAEC0BF0CC0E046FE00E8F
:100EB000056F870E066F050E076FDDEC0CF000C1A5
:100EC0000CF101C10DF102C10EF103C10FF1A2EF4E
:100ED00007F00101800E006F1A0E016F060E026FFF
:100EE000000E036F42C104F143C105F144C106F194
:100EF00045C107F1DDEC0CF003AF83EF07F0B1EC77
:100F00000DF0B5EF07F00E0EDEEC04F0E8CF0CF1BB
:100F10000F0EDEEC04F0E8CF0DF1100EDEEC04F065
:100F2000E8CF0EF1110EDEEC04F0E8CF0FF142C174
:100F300000F143C101F144C102F145C103F107824F
:100F4000EAEC0BF00CC100F10DC101F10EC102F190
:100F50000FC103F10101000E046F000E056F010EB9
:100F6000066F000E076F0BEC0DF077EC0DF01D67B0
:100F7000BFEF07F00401200E826FC2EF07F00401FB
:100F80002D0E826F60EC05F024C182F40401300E56
:100F9000822760EC05F025C182F40401300E82271F
:100FA00060EC05F004012E0E826F60EC05F026C1A6
:100FB00082F40401300E822760EC05F027C182F430
:100FC0000401300E822760EC05F004016D0E826F83
:100FD00060EC05F004012C0E826F60EC05F042C15C
:100FE00000F143C101F144C102F145C103F1010126
:100FF00077EC0DF01EC182F40401300E822760EC04
:1010000005F01FC182F40401300E822760EC05F068
:1010100020C182F40401300E822760EC05F021C16A
:1010200082F40401300E822760EC05F022C182F4C4
:101030000401300E822760EC05F023C182F4040124
:10104000300E822760EC05F024C182F40401300EDA
:10105000822760EC05F025C182F40401300E82275E
:1010600060EC05F026C182F40401300E822760ECAA
:1010700005F027C182F40401300E822760EC05F0F0
:101080000401480E826F60EC05F004017A0E826F55
:1010900060EC05F004012C0E826F60EC05F056C187
:1010A00000F157C101F158C102F159C103F1010129
:1010B00077EC0DF01EC182F40401300E822760EC43
:1010C00005F01FC182F40401300E822760EC05F0A8
:1010D00020C182F40401300E822760EC05F021C1AA
:1010E00082F40401300E822760EC05F022C182F404
:1010F0000401300E822760EC05F023C182F4040164
:10110000300E822760EC05F024C182F40401300E19
:10111000822760EC05F025C182F40401300E82279D
:1011200060EC05F026C182F40401300E822760ECE9
:1011300005F027C182F40401300E822760EC05F02F
:101140000401630E826F60EC05F004012C0E826FC7
:1011500060EC05F056C100F157C101F158C102F130
:1011600059C103F101010A0E046F000E056F000E54
:10117000066F000E076FECEC0CF0000E046F120E01
:10118000056F000E066F000E076F0BEC0DF077EC8D
:101190000DF01EC182F40401300E822760EC05F0D0
:1011A0001FC182F40401300E822760EC05F020C1DB
:1011B00082F40401300E822760EC05F021C182F434
:1011C0000401300E822760EC05F022C182F4040194
:1011D000300E822760EC05F023C182F40401300E4A
:1011E000822760EC05F024C182F40401300E8227CE
:1011F00060EC05F004012E0E826F60EC05F025C155
:1012000082F40401300E822760EC05F026C182F4DE
:101210000401300E822760EC05F027C182F404013E
:10122000300E822760EC05F00401730E826F60ECD3
:1012300005F004012C0E826F60EC05F0B1EC0DF0AE
:101240004CC100F14DC101F188EC0AF06AEC05F0E7
:101250005FEF09F00401630E826F60EC05F004019A
:101260002C0E826F60EC05F064EC09F004012C0E8A
:10127000826F60EC05F0D7EC09F004012C0E826F50
:1012800060EC05F053EC0AF004012C0E826F60EC68
:1012900005F00101F80E006FCD0E016F660E026FB2
:1012A000030E036F79EC09F004012C0E826F60ECE1
:1012B00005F069EC0AF06AEC05F05FEF09F0030154
:1012C0008A6B0790E8EF0AF0D8900E0EDEEC04F07F
:1012D000E8CF00F10F0EDEEC04F0E8CF01F1100EC4
:1012E000DEEC04F0E8CF02F1110EDEEC04F0E8CF02
:1012F00003F10101000E046F000E056F010E066F71
:10130000000E076F0BEC0DF077EC0DF01EC182F4B0
:101310000401300E822760EC05F01FC182F4040145
:10132000300E822760EC05F020C182F40401300EFB
:10133000822760EC05F021C182F40401300E82277F
:1013400060EC05F022C182F40401300E822760ECCB
:1013500005F023C182F40401300E822760EC05F011
:1013600024C182F40401300E822760EC05F025C10F
:1013700082F40401300E822760EC05F004012E0E89
:10138000826F60EC05F026C182F40401300E8227E2
:1013900060EC05F027C182F40401300E822760EC76
:1013A00005F004016D0E826F60EC05F01200120E64
:1013B000DEEC04F0E8CF00F1130EDEEC04F0E8CF31
:1013C00001F1140EDEEC04F0E8CF02F1150EDEECB4
:1013D00004F0E8CF03F101010A0E046F000E056F5F
:1013E000000E066F000E076FECEC0CF0000E046FA1
:1013F000120E056F000E066F000E076F0BEC0DF05E
:1014000077EC0DF01EC182F40401300E822760ECEF
:1014100005F01FC182F40401300E822760EC05F054
:1014200020C182F40401300E822760EC05F021C156
:1014300082F40401300E822760EC05F022C182F4B0
:101440000401300E822760EC05F023C182F4040110
:10145000300E822760EC05F024C182F40401300EC6
:10146000822760EC05F004012E0E826F60EC05F01F
:1014700025C182F40401300E822760EC05F026C1FC
:1014800082F40401300E822760EC05F027C182F45B
:101490000401300E822760EC05F00401730E826FA8
:1014A00060EC05F012000A0EDEEC04F0E8CF00F16B
:1014B0000B0EDEEC04F0E8CF01F10C0EDEEC04F0D4
:1014C000E8CF02F10D0EDEEC04F0E8CF03F188EF77
:1014D0000AF0060EDEEC04F0E8CF00F1070EDEECB9
:1014E00004F0E8CF01F1080EDEEC04F0E8CF02F1E1
:1014F000090EDEEC04F0E8CF03F188EF0AF00101F9
:10150000B1EC0DF007844AC100F14BC101F1079421
:101510000101E80E046F800E056F000E066F000ECD
:10152000076FECEC0CF0000E046F040E056F000E5C
:10153000066F000E076F0BEC0DF0880E046F130E94
:10154000056F000E066F000E076FDDEC0CF00A0E43
:10155000046F000E056F000E066F000E076F0BEC98
:101560000DF077EC0DF001011D67BCEF0AF00401EE
:10157000200E826FBFEF0AF004012D0E826F60EC27
:1015800005F024C182F40401300E822760EC05F0DE
:1015900025C182F40401300E822760EC05F026C1DB
:1015A00082F40401300E822760EC05F004012E0E57
:1015B000826F60EC05F027C182F40401300E8227AF
:1015C00060EC05F00401430E826F60EC05F0120040
:1015D00081A8A6EF0BF007A85FEF0BF00101800ECA
:1015E000006F1A0E016F060E026F000E036F3EC1F0
:1015F00004F13FC105F140C106F141C107F1DDEC45
:101600000CF003BFA6EF0BF0E4EC0BF03EC100F1D1
:101610003FC101F140C102F141C103F10782EAEC8F
:101620000BF00CC104F10DC105F10EC106F10FC1A3
:1016300007F1F80E006FCD0E016F660E026F030EFC
:10164000036FDDEC0CF00E0E0C6E00C10BF0C8EC5D
:1016500004F00F0E0C6E01C10BF0C8EC04F0100E7C
:101660000C6E02C10BF0C8EC04F0110E0C6E03C13D
:101670000BF0C8EC04F007840101B1EC0DF04AC195
:1016800000F14BC101F107940A0E0C6E00C10BF082
:10169000C8EC04F00B0E0C6E01C10BF0C8EC04F0AA
:1016A0000C0E0C6E02C10BF0C8EC04F00D0E0C6EAB
:1016B00003C10BF0C8EC04F00798A6EF0BF007AAE3
:1016C000A6EF0BF007840101B1EC0DF04AC100F167
:1016D0004BC101F10794060E0C6E00C10BF0C8EC73
:1016E00004F0070E0C6E01C10BF0C8EC04F0080EFC
:1016F0000C6E02C10BF0C8EC04F0090E0C6E03C1B5
:101700000BF0C8EC04F0078452C100F153C101F1A1
:1017100054C102F155C103F10794120E0C6E00C1C1
:101720000BF0C8EC04F0130E0C6E01C10BF0C8EC0A
:1017300004F0140E0C6E02C10BF0C8EC04F0150E90
:101740000C6E03C10BF0C8EC04F0079A0401805141
:1017500081197F0B0BE09EA809D014EE00F0815197
:101760007F0BE126E750812B0F01AD6E26EF05F0D0
:101770000CC100F10DC101F10EC102F10FC103F165
:10178000000E046F000E056F010E066F000E076F4E
:101790000BEC0DF01DA1E3EF0BF01451D8B4E3EF07
:1017A0000BF00CC100F10DC101F10EC102F10FC12E
:1017B00003F1000E046F000E056F0A0E066F000E97
:1017C000076F0BEC0DF0120001010C6B0D6B0E6B33
:1017D0000F6B12000101005305E1015303E10253B5
:1017E00001E1002BADEC0CF0B1EC0DF02C51006FD1
:1017F0002D51016F420E046F4B0E056F000E066FE8
:10180000000E076FECEC0CF000C104F101C105F112
:1018100002C106F103C107F10CC100F10DC101F1D4
:101820000EC102F10FC103F107B21BEF0CF0E1ECA6
:101830000CF01DEF0CF0DDEC0CF000C10CF101C15F
:101840000DF102C10EF103C10FF11200B1EC0DF068
:101850004CC100F14DC101F1060EDEEC04F0E8CF01
:1018600004F1070EDEEC04F0E8CF05F1080EDEEC23
:1018700004F0E8CF06F1090EDEEC04F0E8CF07F142
:10188000DDEC0CF000C118F101C119F102C11AF12F
:1018900003C11BF1290E046F000E056F000E066FC9
:1018A000000E076FECEC0CF0EE0E046F430E056FAC
:1018B000000E066F000E076FE1EC0CF018C104F18A
:1018C00019C105F11AC106F11BC107F1ECEC0CF0CE
:1018D00000C110F101C111F102C112F103C113F1F4
:1018E000120EDEEC04F0E8CF04F1130EDEEC04F08F
:1018F000E8CF05F1140EDEEC04F0E8CF06F1150E8A
:10190000DEEC04F0E8CF07F10D0E006F000E016F62
:10191000000E026F000E036FECEC0CF0180E046F5B
:10192000000E056F000E066F000E076F0BEC0DF03A
:1019300010C104F111C105F112C106F113C107F183
:10194000E1EC0CF06A0E046F2A0E056F000E066FB4
:10195000000E076FDDEC0CF01200BF0EFA6E200EC9
:101960002D6F2C6BD8900037013702370337D8B072
:10197000BEEF0CF02D2FB3EF0CF02C072D07035307
:10198000D8B412000331070B8009326F03390F0BF3
:10199000010F2C6F80EC5FF0336F2C0580EC5FF053
:1019A000335D335F2C6B3233D8B02C272C3332A904
:1019B000D3EF0CF033512C271200D6EC0DF0D8B039
:1019C000120003510719286F99EC0DF0D8900751B8
:1019D000031928AF800F1200286BBDEC0DF0D8A0C2
:1019E000D3EC0DF0D8B01200A8EC0DF0B1EC0DF076
:1019F0001F0E296FE9EC0DF00B35D8B099EC0DF006
:101A0000D8A00335D8B01200292FFAEF0CF028B176
:101A1000C0EC0DF01200286B0451051106110711DE
:101A20000008D8A0BDEC0DF0D8A0D3EC0DF0D8B0D4
:101A30001200086B096B0A6B0B6BE9EC0DF01F0EC3
:101A4000296FE9EC0DF007510B5DD8A434EF0DF0D0
:101A500006510A5DD8A434EF0DF00551095DD8A4F4
:101A600034EF0DF00451085DD8A047EF0DF004519C
:101A7000085F0551D8A0053D095F0651D8A0063D75
:101A80000A5F0751D8A0073D0B5FD8900081292F2E
:101A900021EF0DF028B1C0EC0DF0286BBDEC0DF07E
:101AA000D890EDEC0DF007510B5DD8A464EF0DF06C
:101AB00006510A5DD8A464EF0DF00551095DD8A464
:101AC00064EF0DF00451085DD8A073EF0DF0003FF6
:101AD00073EF0DF0013F73EF0DF0023F73EF0DF068
:101AE000032BD8B4120028B1C0EC0DF01200010194
:101AF000286BBDEC0DF0D8B01200F2EC0DF0200E0A
:101B0000296F003701370237033711EE27F00A0E2D
:101B10002A6FE7360A0EE75CD8B0E76EE5522A2F47
:101B200089EF0DF0292F81EF0DF028B11D81D8909C
:101B30001200045100270551D8B0053D0127065178
:101B4000D8B0063D02270751D8B0073D0327120041
:101B50000051086F0151096F02510A6F03510B6F59
:101B600012000101006B016B026B036B120001019B
:101B7000046B056B066B076B12000335D8A01200CF
:101B80000351800B001F011F021F031F003FD0EFF6
:101B90000DF0013FD0EF0DF0023FD0EF0DF0032B21
:101BA000282B032512000735D8A012000751800BFF
:101BB000041F051F061F071F043FE6EF0DF0053F3A
:101BC000E6EF0DF0063FE6EF0DF0072B282B07257B
:101BD00012000037013702370337083709370A3751
:101BE0000B3712001D6B1E6B1F6B206B216B226B62
:0C1BF000236B246B256B266B276B120007
:10BF0000E844F926000C160C2B0C3F0C520C640C68
:10BF1000760C860C960CA50CB30CC10CCF0CDC0C6B
:06BF2000E80CF40C000C1B
:00000001FF
